:1000000009C00EC00DC00CC00BC00AC009C008C09A
:1000100007C006C011241FBECFE9CDBF29D062C0E2
:10002000EFCF26EB33E003C0F9013197F1F70197E9
:10003000D8F70895A39A83E687B986EC86B93699EE
:10004000FECF369A3699FECF85B1089585E089BDF9
:1000500085E090E0E6DF19BC88EC90E0E2CF84E137
:1000600089BD86E990E0DDDF19BC88EC90E0D9CF4E
:1000700082E087BB81E28FBD81E083BF81E687B9E3
:10008000A29A86EC86B9479AD5DFE82EF12C3798EC
:10009000BB9AC39A00E010E003C0E1DF04561109E7
:1000A000E801CE0DDF1DC436D105B8F788EE93E028
:1000B000B8DFCA30D10520F4C9DF02C02A97CFDFEC
:1000C000CA30D105D8F788EE93E0ABDF209721F452
:1000D000BDDF02C02197C3DF2097E1F788EE93E0F0
:0800E000A0DFFCCFF894FFCF74
:00000001FF
